:020000040000FA
:060000000219FD020310CD
:03001300020501E2
:03001B0002008D53
:03002B000202D5F9
:03005B000205108B
:030073000202FD89
:100080000406080C10182030406080A0C0C2AFC227
:10009000A853E6EFC28E856B8BC0D0D2D3C0E0C030
:1000A000F0C2CAA8CCA9CDD2CAD2AF758A00C3E823
:1000B000956CF8E9956DF9C3E913F9E813F8E5666D
:1000C0006007C3E913F9E813F8E97025E8956E4075
:1000D00020956E501CE582B410177C007B007A00DE
:1000E0007908900000A86AE5667004C3E813F80177
:1000F000FA900000D2A8D2AA61BAE0FDC39CC398CE
:1001000040EF98EB33FB0582E0FCC39DC39840E1D0
:1001100098EB33FB0582E0FDC39CC39840D398EB7A
:1001200033FB0582E0FCC39DC39840C598EB33FBCD
:100130000582E0FDC39CC39840B798EB33FB058272
:10014000E0FCC39DC39840A998EB33FB0582E0FD1A
:10015000C39CC398409B98EB33FB0582E0FCC39D96
:10016000C398408D98EB33FB05822175900000D237
:10017000A8D2AA61BAE0FDC39CC39840EF98EA33C5
:10018000FA0582E0FCC39DC39840E198EA33FA0582
:1001900082E0FDC39CC39840D398EA33FA0582E01D
:1001A000FCC39DC39840C598EA33FA0582E0FDC3BD
:1001B0009CC39840B798EA33FA0582E0FCC39DC31C
:1001C0009840A998EA33FA0582E0FDC39CC39840A1
:1001D0009B98EA33FA0582E0FCC39DC398408D9852
:1001E000EA33FA0582EBC46B6A54F0F9EAC454F0BE
:1001F000C3996009900000D2A8D2AA61BAEBF4C4F6
:1002000054F0F9EAF4C4540F49FAEBF4C4540FFB68
:10021000C3EAF99460FAEB9400FB5020C3E97B0039
:100220007A0079006016C3135006F9C39552600A2C
:10023000E9F552755300790080020553303A27C31F
:10024000EA94D0F8EB9407F9400BE8FAE9FB203583
:1002500009D235415A303502C235203902B235C390
:10026000EA33FAEB33FBEB2B3B3BF9C3EB13FBEA33
:1002700013FAEA29FAEB3400FB30E3047AFF7BFF40
:10028000E5255403601B202A18E55D33F9EB700760
:10029000C3E99A4002E9FAE53CC4332AFAEB340098
:1002A000FBC3EA33C4540FF8EB33C454F048F8707E
:1002B00005EA60027801C3EB13FBEA13FA90000031
:1002C000D2A8D2AAE52260021522819E900000D217
:1002D000A8D2AA61BAC0D0C0E0C2CF0541E5236070
:1002E000021523C3E554600575550041F8E5552412
:1002F00001F55550037555FFD0E0D0D032C2AF5351
:10030000E67F7592FA7593FFC22053917FD2AF3288
:10031000C0E0E58A303408856B8BF0A3D0E032D0A2
:10032000E0C2AF53E6EFC0D0C0E0C0F0D2D3D2AF4E
:100330005388EFA88AA98C758A00758C00438810B1
:1003400030331FE8C4540FFAE9C454F04AFAC31317
:100350002AFAC3E833F8E933F9E82AFAE93403FB67
:1003600061AB30320FC3E833E933FAE82AFAE934F3
:1003700000FB61AB303115E875F056A4AAF0E975C1
:10038000F056A42AFAC5F03400FB61ABE875F02BF7
:10039000A4AAF0E975F02BA42AFAC5F03400C3131F
:1003A000FBEA13FAC3EB13FBEA13FAC3EB9409500D
:1003B00009C3EA949AEB940350160522E5227002D1
:1003C0001522C3E5229432500281F475540081F75E
:1003D000E522600215223036067C007D0461EAAC1D
:1003E00031AD32303A04AC33AD34C3EA9CFAEB9D04
:1003F000FB9208AE60AF61303A425007203509D217
:10040000358108303502C235303504AE62AF632025
:100410003902B235C3EA33FAEB33FBA208500AEAD9
:10042000F42401FAEBF43400FBC3EA9428FAEB94C9
:1004300000FB501478007A007B008148A208500825
:1004400078007A007B00819EE52554036019202AFC
:1004500016E55DF9EB7007C3E99A4002E9FAE53C5D
:10046000C42AFAEB3400FBEA8EF0A4F9AAF0EB8E72
:10047000F0A42AFAC5F03400FBC3EB13FDEA13F82D
:100480000FEF146004C3E833F8C3E933EA33FAEB3F
:1004900033FBDFEDEB30E20678FF7AFF7B03885415
:1004A000D230E86003755500C3E55BFC955C400203
:1004B000AC5CC3EC95545008EC75F004A4FAABF0B6
:1004C000EAF4F8EBF45403F98856895775230AE5E2
:1004D0005A30E110D0F0D0E0D0D053F7DF43F740EE
:1004E00043E61032D0F0D0E0D0D053D8FE43DA014A
:1004F00043E6103275230AD0F0D0E0D0D043E610A6
:1005000032C2AAD28EC2CA85CC6C85CD6DD2CA3217
:10051000C2AFC0D0C0E0D2D38556FB8557FC85570B
:100520005A53F7BF53DAFED2A8303402D2AA53E6A8
:10053000EF53F7DF53D8FED0E0D0D0D2AF327901FD
:10054000801479038010790A800C791E8008796400
:10055000800479C880007817E4D5E0FDD8FAD9F690
:100560002278FF20282879A1E76023E548601F74DE
:10057000FF8548F084853FF030290375F005A4F825
:10058000C5F0600278FFC3E8955D5002A85D885C05
:1005900022C3E54794E4E5489400E55C500314A1C8
:1005A000A2046002F55C2275E89022055EC3E55E58
:1005B0009408405330EDF4A8BDA9BE755E00E9FA79
:1005C00079A0E76041EA7006E55F6018800CC3E837
:1005D000955F600EE55F5005600A1480070460FABD
:1005E0008002E55FF55FC39569401B755BC0C394EE
:1005F000044013755B80C39404400B755B40C39447
:10060000044003755B0022E55B2410500274FFF583
:100610005B22743279A687F0A4C5F0A2F733F55DAA
:10062000227547007548F022C2AFC2CAA8CCA9CD36
:10063000AA4130CF010AD2CAD2AFAB42AC43884202
:100640008943C3E89BF8E99C202808F9302C02E193
:1006500038C191AD448A44F9EA9DFA600678FF7981
:10066000FFC176AE45AF468B458C46A842A943C331
:10067000E89EF8E99FF9C3E54813FBE54713FAE85C
:100680002AF547E93BF54850067547FF7548FFC115
:10069000DEAA47AB48AC47AD487E047F02C3EB946B
:1006A00004400D1E1FC3EB940840052029021E1FA5
:1006B000C3ED13FDEC13FCDEF7C3EA9CFAEB9DFBE4
:1006C000EF6009C3E913F9E813F8DFF7EA28FAEB5A
:1006D00039FB8A478B4850067BFF8B478B48C3EB1F
:1006E00094025002D22C3028047F03E1097892E66C
:1006F000FFC3E53D948240110FC3E53D94A0400146
:100700000FC3EF940640027F057E02E548C4540FF4
:10071000F9E548C454F0F8E547C4540F28F8C3E895
:100720009EFAE99400FB4009C3EA9401EB9400505F
:10073000047A01E4FB020784AA47AB48EBC4FEEA53
:10074000C4540F4EFCC3EA9CFAEB9400FBC3E813BD
:10075000C313F8EA28FAEB3400FB8A478B48C3EB53
:1007600094024002C22C7802EBC4FE7B00EAC4541F
:100770000F4EFAC3EA98FA4005C3940150027A0179
:100780007892E6FF302002E184854E92854F93D225
:100790002043E680C3E49AF8E49BF9302C03020876
:1007A00012E8FAE9FBD3E913FDE813FC884E894F00
:1007B000C3EF94036038EF20E00CE82CF8E93DF932
:1007C000ECFAEDFB8013E828F8E939F9C3E82401D5
:1007D000F8E93400F97AFF7BFFC3EF9403400F8AF6
:1007E000508B51884A894B8C4C8D4D02084788505C
:1007F00089518A4A8B4B8C4C8D4D3028127550F0A4
:100800007551FF754CF0754DFF754EF0754FFF0239
:100810000847E8FAD3E813FC884EC3EF940360213D
:10082000EF20E007E82CF8ECFA0132E8282401F880
:100830007AFFC3EF940340098A50884A8C4C02081F
:100840004788508A4A8C4C3020020147753A02D2C0
:100850002043E680E52554036034A847A948C3E94E
:1008600013F9E813F8C3E913F9E813F8302804E999
:100870002440F9C2AF53E67F759100C3E498F59424
:10088000E499F595759104D22043E680D2AF22D247
:1008900021754900752000302B0375204001ADD231
:1008A00021754900752040302B03752000780179AF
:1008B00001202C20E52554036002C2217914E5486B
:1008C000C313700104F8C394144002781430280450
:1008D000781B791B202010E549600C302803D53A9D
:1008E00004D2222154114F0549E59B5440B5200202
:1008F000213E30280908C3E89940011801D420217D
:100900000A08C3E899400201AD01D4C22153E67F31
:10091000759100302C117594007595F8759104D27D
:100920002043E6800208ADE5487EFFC3334005C39F
:10093000334001FEC3E49E759400F595211CC3E588
:10094000399401500201AD30210201ADD80221528B
:1009500001D4C222C2AF53E67F75910085509485C1
:100960005195759104854A92854B93D22043E68038
:10097000D2AFE525540360072029020539801030E5
:10098000220D202B0A20210715811581021399229F
:1009900078003021027801E53D75F007A4F9E5F013
:1009A00028F5F0E9A2F013A2F113A2F213F53DC36A
:1009B00094785003753D78C3E53D953E400CC29553
:1009C000C291C28775D4FF75D57F30200221CA85B8
:1009D0004C92854D93D22043E68022203817C2AF37
:1009E000C291C296D295D28775D4FF75D57FD2AF0A
:1009F000759F1241FFC2AFC291C290D287D2957546
:100A0000D4FF75D53FD2AF759F1241FF203817C272
:100A1000AFC287D29175D4FF75D56FC296D295D2E9
:100A2000AF759F3241FFC2AFC295D29175D4FF75A9
:100A3000D56FC290D287D2AF759F0241FF20381781
:100A4000C2AFC295C290D287D29175D4FF75D56FCF
:100A5000D2AF759F0241FFC2AFC287C296D295D274
:100A60009175D4FF75D56FD2AF759F3241FF203895
:100A700017C2AFC291D29575D4FF75D53FC290D23F
:100A800087D2AF759F128077C2AFC291D28775D4DB
:100A9000FF75D57FC296D295D2AF759F1280602028
:100AA0003817C2AFC287C294D291D29575D4FF7560
:100AB000D53FD2AF759F328046C2AFC295C294D2A5
:100AC00091D28775D4FF75D57FD2AF759F02802FE5
:100AD000203817C2AFC295D28775D4FF75D57FC2B3
:100AE00094D291D2AF759F028015C2AFC287D295C2
:100AF00075D4FF75D53FC294D291D2AF759F322283
:100B00007A147B7880127A107B8C800C7A0D7BB4FF
:100B100080067A0B7BC88000E564D5E0012279026B
:100B2000E4C291D5E0FDD294D291D5E0FDC291D539
:100B3000E0FDC294D291D5E0FDE920E004D296D246
:100B40009530E004D290D287E564D5E0FDE920E05D
:100B500002C29530E002C2877496D5E0FDD9C1EAA1
:100B6000F8D5E0FDD8FBDBB0C29122C295C291C29C
:100B700087C295C291C28775D4FF75D57F227880D0
:100B800076FF0876FF0876FF0876FF0876FF08767E
:100B9000FF0876090876FF087601788C76010876DA
:100BA000FF0876FF0876FF0876FF0876FF087603D1
:100BB0000876FF0876FF0876FF0876250876D008C5
:100BC00076280876500876040876FF0876020876BC
:100BD000FF08767A0876FF0876070876010876FF20
:100BE0000876FF08760008760022FA75F00CA4ABB0
:100BF000F0EAC333F8740133F9E8C333F8E933F9A1
:100C0000E8C32BF8E93400F9227888E6C39403D2CC
:100C10003A5002C23AC238E630E102D238A23892E3
:100C2000397886E6149000809378A6F67886E6F503
:100C30003FC394025003753F02789CE6753EFFB4B3
:100C40000203753EA0B40303753E8278A0E6F86007
:100C50000674282409D8FCF5697896E671EA88318B
:100C60008932789EE671EA883389347897E671EAAA
:100C700088358936716B223036117A007B007CFF13
:100C80007D007E0091DD8B618A6022303A22789669
:100C9000E6FA7B00789EE6FC7D00C3EA33FAEB338C
:100CA000FBC3EC33FCED33FD7E0A91DD8B638A627E
:100CB0007896303A02789EE6FA7B007897E6FC7DDB
:100CC000007E00303A10C3EA33FAEB33FBC3EC3357
:100CD000FCED33FD7E0A91DD8B618A6022C3EC9EC0
:100CE000FCED9400FDC3EC9AFCED9BFDC3EC94235A
:100CF000ED940050047C237D00C3EC94FFED94013F
:100D000040047CFF7D017BFF0B7A000AEA7009C377
:100D1000EC33FCED33FDA108EC8AF0A4AEF0ED8AD3
:100D2000F0A42E947C40E4EAF460DD22D236917780
:100D300012054A12054A7A007B007C10120542E532
:100D4000542AFA74003BFBDCF37C04C3EB13FBEA8C
:100D500013FADCF7FFEB60027FFFC236917722784F
:100D6000A5E6F954037000E9540C7000E9543070A2
:100D700000E954C07000227567007568007597DE41
:100D80007597AD7581C043FF8075EF0675A9007139
:100D90006B75807F75F1F075A48075807F75D4FFC9
:100DA00075900075F27375A57375900075D57F7594
:100DB000A60175E34075E202716BE4F8F6D8FD71A7
:100DC0007E1213D478988664753001C2AF12055232
:100DD000710012054A710612054A710C12054AB1DA
:100DE0005FC2AF75670075680078FA79FA308507D9
:100DF000D9FBD8F7021C0091099177789886647125
:100E00006B75E405758811758E0475890975C804BC
:100E100075910475D84075D90875F782759E00756F
:100E2000960075DA4A75DB0075A82175E69075B8ED
:100E300001759B80759D0075D10C75BC5975BB10F3
:100E400075E88075B20112053ED2AF753C00C23024
:100E5000120552C231C232C233C2347552007553C8
:100E60000075220012054EC3E522940A5002E138B3
:100E7000D23175220012054EC3E522940A5002E1D8
:100E800038C231D23275220012054EC3E522940ACF
:100E90005002E13875E4D5758851758E017589AABF
:100EA000758C00758D00C2A9D2ABD2AA756BC075C6
:100EB0006A14756E50C232D23475220A12054E750C
:100EC0006A10C3E522940A75520075530040697593
:100ED0008E0C756B80756A28756E2875220A12054E
:100EE0004E756A20C3E522940A755200755300407E
:100EF00047758E0C756BC0756A14756E1475220A71
:100F000012054E756A10C3E522940A755200755396
:100F100000402575E405758811758E04758909D220
:100F2000A9C2ABC2AAC234D23375220012054EC385
:100F3000E522940A4002A1E1120542203003020D8D
:100F4000E1C2AF710071007100D2AF1205522034BE
:100F500003303A03020FF8120542788CE6C394017D
:100F60005003020FF8E530C394015003020FF875E7
:100F700067A57568F17F02D236917712054EC2AF30
:100F8000C2369177C3E554947FD2AF406B12053ED1
:100F9000C2AF7112D2AFDFDFB12CC3EF7897F61278
:100FA00005521214C17F0AD236917712054EC2AF94
:100FB000C2369177C3E554947FD2AF50E812053E14
:100FC000C2AF71001205467100D2AFDFDAB12CEF6B
:100FD00024037896F6F87997E7C394234003985052
:100FE00006E824237897F612055212141B1214F007
:100FF00012054E9177020DE17567007568001205C4
:101000004EC3E55494014003020F4EC2AF120B12BF
:10101000120B12120B12D2AF120552753000E4F50A
:1010200037F5380537E537F4703F0538789AE678B4
:1010300019146012783214600D787D14600878FA03
:10104000146003753800C3E53898401D120B6B120D
:10105000053E153875370078998664C2AF120B12B9
:10106000D2AF7898866412054E120546E5237003C8
:10107000020DE1C3E5549401500AC3E552940150B6
:101080001602102312054EE5237003020DE175527E
:1010900000755300021239C3E55294017017C2AFB4
:1010A000120B6B78998664120B0078988664D2AF25
:1010B00012054E412BC3E55294027017C2AF120BBA
:1010C0006B78998664120B0678988664D2AF120505
:1010D0004E412BC3E55294037017C2AF120B6B78CD
:1010E000998664120B0C78988664D2AF12054E4133
:1010F0002BC3E55294047017C2AF120B6B7899861C
:1011000064120B1278988664D2AF12054E412BC33D
:10111000E55294057017C2AF120B6B789986641272
:101120000B1278988664D2AF12054E412BC3E5525C
:1011300094077019C3E5539406500201737401308B
:101140003A0274037888F6C238C239412BC3E5529B
:1011500094087019C3E55394065002017374023069
:101160003A0274047888F6D238D239412BC3E5525A
:1011700094097017C3E553940650020173303A0B7B
:10118000C37888E69402F6C23A412BC3E552940A2A
:101190007016C3E553940650020173203A0A78880A
:1011A000E62402F6D23A412BC3E55294147025C3CB
:1011B000E553940650020173C2AF901A0B7400936A
:1011C000D2AF7888F613C238C2394002D238400212
:1011D000D2398057C3E55294157038C3E55394064D
:1011E000404FC2AF901A0B740093D2AFF8B801020F
:1011F0007402B802027401B803027404B8040274E1
:10120000037888F613C238C2394002D2384002D27D
:10121000398018C3E552940C70117567A57568F193
:10122000C3E5539406400A911BD2AF755200755323
:10123000007567007568000173C2AF120B6BE4D2D2
:10124000AFE4F55EF524F525F53D755E0812053E23
:101250001205A730EDFDA8BDA9BEE97001F8885FB1
:101260001205AB755E08C2AF120612855D5B855D27
:101270005CD2AF303A07C238303502D238D2287546
:101280003900120A9F120AD01206211206281206ED
:101290002112062812062112089F1209901209DB5A
:1012A00012062812088F202C03120561302C03121D
:1012B0000591120990120A0C12062812089F1209B1
:1012C00090120A3D12062812088F120990120A6E17
:1012D00012062812089F120990120A9F120628125D
:1012E00005A712088F120990120AD01205AB120638
:1012F00028302827855D5B79187A0CC3E539994039
:101300000EC228D2298A3B855D5B855D5C800CC35B
:10131000E5549401400302129761A130291F202B4C
:101320001CE53B147006C229D22A4197F53B203AAE
:1013300007C3E554940140030212978064753C0092
:10134000203A0F78FA79A4E760027803C3E555984C
:10135000504FE523604B303A172038052035078081
:101360000F303502800A202B07D22B855D5B41C7E9
:1013700078F0302B05855D5B7820C3E548985003F5
:10138000021297302B1BC22BC238303502D238D212
:1013900029753B12855D5B4197053CE55460026110
:1013A000A4753C00C2AF120B6B752400752500D2EA
:1013B000AF12054E120B6B78A4E6600CC296D29564
:1013C000C294D291C290D287C3E53C9404400302F8
:1013D0000DE1011E901A0D78209154E520B4550AB4
:1013E000A39154E520B4AA0280137567A57568F12E
:1013F000120B7E911B756700756800801D901A03A3
:1014000078807B0A9154A308DBFA901A0F788C7BC2
:101410001A9154A308DBFA901A2922C2AF9197912E
:1014200074901A0074109159A374079159A37421F0
:101430009159901A0378807B0A9158A308DBFA909F
:101440001A0F788C7B1A9158A308DBFA91AA91881D
:10145000901A2922E493F622E6438F01538FFDFF71
:10146000C3E583941C400122EF8567B78568B7F018
:10147000538FFE22438F02438F018567B78568B77C
:10148000901A0DF0538FFC22901A0D7455915990BB
:101490001A0E74AA9159227A3079D07820901A4085
:1014A0009154E520F709A3DAF7227A3079D0901A1F
:1014B00040E7915909A3DAF9227C05120552DCFBB9
:1014C00022C2AF120B00120B06120B0C120B1212DF
:1014D0000546120B00120B06120B0C120B12120512
:1014E00046120B00120B06120B0C120B12D2AF227B
:1014F000C2AF120B12120B0C120B06120B001205CC
:1015000046120B12120B0C120B06120B00120546A0
:0F151000120B12120B0C120B06120B00D2AF2291
:1019FD00020D77100721FFFFFFFFFFFF09FF01FF1A
:101A0D0055AA01FFFFFFFFFF03FFFFFF25D0285061
:0D1A1D0004FF02FF7AFF0701FFFF0000FF3A
:101A400023565F4C5F303023202020202020202090
:101A500023424C48454C492445464D3842313023B9
:101A60002020202020202020202020202020202076
:101C0000C2AFC2D37597DE7597AD7581C075A90057
:101C100043FF80752438752503B1DB7529A5752A26
:101C2000F143F12053A4DFD28575D4FF75E3407DE5
:101C3000FA780379E67C10752200752300901DE880
:101C40007B0675249875250130850281482085081A
:101C5000D8FBD9F9DCF781BA308508D8FBD9F9DC93
:101C6000F781BAB19BE493A3C39A6004DDC381BA40
:101C7000DBDBB18D600281317B08E493FAA3B16EA6
:101C8000DBF87A30B16E752200752300B18DEAFC65
:101C9000EBFDC3ED94FE400EB18D8A278B28ED300D
:101CA000E0048A828B83B18D7AC270D8C3ED94FE32
:101CB000601950CEBD0029EC600F7520007521FF22
:101CC000752900752A000200008100A827A92808AC
:101CD00009D804D90281DDB191EAF281D10D81A642
:101CE000C3ED94035051EDA2E092007AC5C3E582A2
:101CF0009400E583941C508C200010438F02438F86
:101D0000018529B7852AB7F0300027A827A9280818
:101D100009438F01538FFDD804D902A132C3E58353
:101D2000941C4003A3A117E28529B7852AB7F0A325
:101D3000A117538FFC81827AC1BD030CE493A3FAEF
:101D4000B152DCF8B14A81828184AA22AB23B16E00
:101D5000EBFAEA6222752608C3E52313F523E52290
:101D600013F52250066323A0632201D526EAB1DBD6
:101D7000B1DB75260AEAF4200102D285300102C2E5
:101D800085B1DBC3134002C201D526EB22B191EA33
:101D9000FB208502A191308502A196752608AE240C
:101DA000AF25C3EF13FFEE13FEB1DFB1DBC3EA13C0
:101DB0003085024480FA30E703632201C3E5231330
:101DC000F523E52213F52250066323A0632201D5F3
:101DD00026D9E52265236523F52222AE24AF250E00
:101DE0000FDEFEDFFCD20122424C48656C693437BD
:061DF0003164E8B10601B8
:00000001FF
